:020000020000FC
:100000004CC0FFB6989B38C01123B1F4B29B28C0F6
:020010000AC024
:10001600FFB6112789B3807F8BBB80E083BF36C0D4
:10002600962CA72CB82C662477248824CC24DD248F
:10003600EE24B29B07C0139590E093BF9EEC92BF4F
:1000460093E093BF123058F061F0143018F029F4A1
:100056009B2D08C09091690005C0992703C0992D72
:1000660001C09A2DB29992959F7089B3807F982B83
:1000760008C099B3907FB29B03C08FEF9F6002C008
:100086009229812D9BBB88BB92E0B29B93E095BFE2
:10009600FFBE189521E02EBF2FE52DBF2FEF2ABBFF
:1000A6002BE027BB20E42BBF21E029BFAFD362E0C2
:1000B6007BD263D2F89463E077D22FEF28BB2BBBB9
:1000C6005CD2222723BB20936800ADD380F360E087
:1000D60061F96AD200FDE0D001FDF5D002FD4CD1F8
:1000E60004FDE1D005FDFDD0202F2295022B6624CC
:1000F6007724882455243324442413D093E095BFD1
:10010600789442D2889400FD36D040F001FD43D069
:1001160028F002FD20D010F004D0F2CF2E3081F767
:10012600C9CF98990BC0242D6FEF26272F70222E4A
:1001360069B3607F262BB29B2BBB03C06C2C7D2C36
:100146008E2C232D25296FEFB29968BB2627B29BEB
:1001560028BB122E089520916E002A9519F020933F
:100166006E00089520917E0020936E0097D2C8F30A
:10017600C1F3D0D121C020916E002A9519F02093A9
:100186006E00089520916C0020936E0087D2C8F30C
:10019600C1F38DD111C020916F002A9519F02093DB
:1001A6006F00089520916D0020936F0072D2C8F3FE
:1001B600C1F32093790003D0989488940895989A6F
:1001C6002091680021FD9898B0E0AEE822E0999968
:1001D6002D91233008F008952D91662720FD626049
:1001E60021FD6160562E2695269520613AD02093F2
:1001F600690020917900263030F09B992D919C99C9
:1002060011C09A9918C0CD90DD902D91219529D0D5
:10021600E22E2C2D219525D0C22E2D2D219521D0D3
:10022600D22E08956D912D9129D0C62E6D912D91C6
:1002360025D0D62EEACF6D912C912F7023FD206FFD
:100246001DD0C62E6D9162956F705C915295507F50
:10025600652B2D9122952F7023FD206F0FD0D62E62
:10026600D4CF222351F0622F2A7A60FD246062FDEA
:10027600216064FD206466FD2061089527FD06C0A7
:10028600222311F467FF08956FE708952F3F11F4B5
:1002960067FD089560E808953091750020917C000F
:1002A60050917E0006C03091760020917D005091DD
:1002B6007F003093770020936A0050936C00509330
:1002C6006E0020E0EFC020917C0020936B0020910F
:1002D6007E0020936D0020936F0060918000FED118
:1002E6000DC020917D0020936B0020917F0020930C
:1002F6006D0020936F0060918100EDD109F00895A3
:1003060050917400A6E8B0E05523F9F05A952D9166
:10031600253821F4999A5A952D91F6CF253931F43D
:100326005A952D91203181F79B9AEECF253739F4D6
:100336005A952D91203131F02C3031F0E5CF06D091
:1003460019F308959C9A08959A9A0895237081F056
:100356002A9559F02A9531F05A9561F02D915A95C2
:1003660049F02D915A9531F02D915A9519F02D910C
:100376001894089598940895209175002093770015
:1003860020917C0020936A0020917E0020936C00CF
:1003960020936E0060918000A1D109F00895E2E7F4
:1003A600F4E06AD029F0E8E7F4E066D009F00895B1
:1003B60033273093820030938300309384005A951C
:1003C6002D91253831F433955A952D91209385003A
:1003D600F6CF213A21F45A952D91223011F09894B6
:1003E60008955A952D912537D1F75A952D91283094
:1003F600B1F75A952D91253719F1253911F40CD0FD
:10040600F8CF293011F40BD0F4CF213811F411D0E4
:10041600F0CF9CDF71F308955A950D9008955A9583
:100426002D910A943395203309F008953093820074
:1004360008955A952D91213009F00895300D0895AB
:100446005A952D91213019F0243059F008955A9576
:100456002D91253909F008955A952D91243009F0EA
:1004660001C030683093830018940895050109048B
:10047600A10105010905A10150917400A6E8B0E0AB
:1004860036E005902D91201519F45A953A95C9F73D
:10049600089560918800693309F0089562E020911B
:1004A600680026272093680021FD9898B4C0F1DFE4
:1004B600B0E0A6E860E02C912F7009F062E02D9183
:1004C600207F09F061E0362E2D913327662708D06C
:1004D600622BAE38E0F3462E232D232B322E0895C1
:1004E6005D912227583591F05A3291F05C3271F0C5
:1004F60028E05F5451F021E05A9539F022E05A95F0
:1005060021F024E05A9509F02227089532600895D3
:1005160031600895209182002A95B0E0A6E8A20FE6
:1005260066272D91203009F461602F3F09F4686039
:100536002D91203009F464602F3F09F46260462E45
:1005460020918300622F6F77A6E8A60F6D915C91CC
:1005560027FF08C0569567955695679556956795F2
:1005660056956795562F52956795652B222760FD00
:10057600226061FD2160322E089532E303D03A9560
:10058600E9F7089544E601C04AE003D04A95E9F741
:10059600089524E6000000000000000000002A95EF
:1005A600C9F7089523E0F6CF78EA7260DF987FB93D
:1005B60020D06FB91ED0DF9A08957260DF987FB998
:1005C60018D02D9115D05A95E1F7DF9A0895DF9846
:1005D6007FB90FD0222715D0DF9A0895DF987FB90B
:1005E60008D022270ED02D935A95D9F7DF9A089571
:1005F6002FB920E42EB93BE13DB92EB126FFFCCF41
:1006060008952FB920E42EB93BE13DB92EB126FF5E
:10061600FCCF2FB10895F9E0E4E861E08BD170E2F8
:1006260058E0CBDF60E478EEC0DF20E12093700075
:10063600B4D009F0089560E878EEB7DF222720935A
:1006460071002093720003C060E078E3AEDF609132
:10065600680070E1AADF61E078E3A7DF20E220937B
:100666007000C6D009F40895243041F42091710039
:10067600239520937100283C39F709C02E3039F4B0
:10068600209172002395209372002530E9F62223EB
:100696000895AEE8B0E020916B0004C0A6E8B0E093
:1006A60020916A0020937000A3D029F0243011F025
:1006B60008940895089570E38ADF522F2F9378E007
:1006C60086DF2D935A95D9F778EC64E06EDF2F918B
:1006D600222388940895F9E0E4EA09C0F9E0ECE9F8
:1006E60006C0F9E0E4E903C062E1F9E0ECE822D1F2
:1006F60070E258E062DF20E1209370004ED009F0EE
:10070600089578EE60E260937A004FDF2E912E9185
:1007160006D021F420EA209370003FC00895A6E891
:10072600B0E02093780022272093740020E02093E5
:10073600700033D009F0089570E349DF2093730009
:10074600522F78E044DF2D935A95D9F778EC64E080
:100756002CDF2091740050917300250F20937400B4
:1007660020917700521730F0209174005091780054
:100776002517E0F222270895F9E0ECE7DAD0A0E6A3
:10078600B0E070E258E019DF20E12093700005D058
:1007960009F0089520E82093700022272093710025
:1007A6002093720025D009F40895243041F4209155
:1007B6007100239520937100283CA1F709C02E30C3
:1007C60039F420917200239520937200253051F759
:1007D600263061F460917A00603111F060E101C069
:1007E60060E260937A0078EEE0DEE1F62223089577
:1007F6006091700070EFD9DE78ECE9DE2078E1F3E5
:1008060060E8D3DE78EFE3DE2F70089578E864E1E0
:10081600CCDE78E760E2C9DE60E0C7DE78E6D7DEE8
:100826002170E9F308953DD0D0F158EC90D054D022
:10083600B1F55ADFA1F568E054DF89F560918800CB
:1008460050DF30918A00EFE8F0E00781002309F4D9
:1008560004E020892093800024892F7020937C0057
:10086600268920937500208D20937E003130A1F0DB
:10087600043091F0E8EAF0E027812295022B2089E6
:100886002093810024892F7020937D002689209350
:100896007600208D20937F006FDF8894089508945A
:1008A600089578ED61EC81DE78EC60E27EDE78EE2C
:1008B60064E07BDE78EF8BDE207C61F078ED20381B
:1008C60021F06BEC72DE689403C069EC6EDEE8948E
:1008D600889408950894089528E02093770078EE88
:1008E60061E063DE78EE73DE2170E1F758EC2FD01D
:1008F60060E070EE5ADE68E0F8DE09F008952091B7
:100906008D002093770078EE61E04FDE78EE5FDEB3
:100916002170E1F758EC1BD0F9E0ECE62FDF09F087
:1009260008955EE114D061E070EE3FDEF9E0E4E7A1
:1009360025CF662767FD60E807D058E025912D93FF
:100946005A95E1F75E936E93B0E0A0E6089578ECD1
:1009560060E42BDE78EC3BDE2074E1F360E425DE18
:100966005A95C1F70895000501000000000000092E
:10097600010000000000210A00000000000021091B
:10098600000200000100800600010000120080063F
:10099600000200008000810600220000800081061F
:0609A600002201008000A8
:100FC0004D535848494431207665722E322E3720D1
:100FD0002020202031322E30332E323032310D0A93
:100FE000415454696E7934342F3834202020202025
:100FF000202020202020286329206361726F0D0AA1
:00000001FF
